:100000000C942A000C94310A1895000018950000F1
:10001000189500001895000018950000189500002C
:100020001895000018950000189500000C947200B7
:10003000189500000C943A0B1895000018950000D4
:1000400018950000189500001895000018950000FC
:10005000189500008FE58DBFC0E4E8E34E2E88E0E0
:100060008EBFD8E0F8E05F2EEEEFF7E0A0E6B0E05C
:10007000A89584B7082E877F84BF88E1992781BD22
:1000800091BD88278D933197E9F789E089B980E0A0
:1000900080BD88E18AB966240E94520C8D9A8C9AA0
:1000A00083EF8FBD83E08EBD8FEF93E090934B0085
:1000B00080934A008FEF84BB8E9A8F9ABB9ABC9A2A
:1000C0008A98929A85B78C7F826085BF8BB780644F
:1000D0008BBF83B7816083BF89B7816089BF8EE69C
:1000E00082BF41C00F938F938FB78F93AF93BF930E
:1000F0009F93A2E6B0E08D919C9101969C938E9384
:1001000000278130900731F4AA9AAB9AAE9AAD9A43
:10011000C09A1FC0903041F0803D07E09007C8F0C2
:1001200000270D930C9315C012969D91891708F026
:10013000AA989D91891708F0AB989D91891708F0AE
:10014000AE989D91891708F0AD989D91891708F098
:10015000C0988EE682BF9F91BF91AF918F918FBF64
:100160008F910F91189587E886B980E487B9579ADF
:10017000E5E0F0E0A5E8B0E00E94210CE6E0F0E068
:10018000A6E8B0E00E94210CE7E0F0E0A7E8B0E0CC
:100190000E94210CE8E0F0E0A8E8B0E00E94210C09
:1001A000E2E0F0E0A2E8B0E00E94210CE3E0F0E041
:1001B000A3E8B0E00E94210CE4E0F0E0A4E8B0E0A5
:1001C0000E94210CE0E0F0E0A0E8B0E00E94210CE9
:1001D000E1E0F0E0A1E8B0E00E94210C0091850090
:1001E0000C3818F011F00C94F7000C9403018BE418
:1001F000809385008BE4809386008BE48093870056
:100200008BE48093880080918500809364008091C6
:1002100086008093650080918700809366008091BE
:100220008800809367008091820080936800379AED
:10023000789480E180934101AAE8B0E088278C930C
:10024000C498C39889B78E7F89BF0E94CF0A082FB0
:10025000013011F00C943101AAE8B0E038E00E94BE
:10026000B60AAAE8B0E0EAEAF8E10E943B0C11F015
:100270000C943C010C943E010C94250189B78160DB
:1002800089BF80E293E0A3E9B0E08D939C93ADE752
:10029000B0E00E94660B8DE00E940B0BE0EBF8E1F2
:1002A0000E94010B0E94080B8FEF93E090934B008C
:1002B00080934A00009185000C3818F011F00C94DE
:1002C00063010C946F018BE4809385008BE4809331
:1002D00086008BE4809387008BE480938800809174
:1002E00085008093640080918600809365008091F2
:1002F00087008093660080918800809367008091DA
:1003000082008093680080E080933B0180E08093CE
:100310003C010E94CF0A082F013011F00C94AB056C
:10032000AAE8B0E038E00E94B60AAAE8B0E0E6EC3D
:10033000F8E10E943B0C11F00C94AD01AAE8B0E08A
:1003400038E00E94B60AAAE8B0E00E94DB0BA3E9FD
:10035000B0E00D931C930C94AB05ECECF8E10E941B
:100360003B0C11F00C94BE0182B390E4892782BB50
:1003700082B390E8892782BB0C94AB05E0EDF8E1ED
:100380000E943B0C11F00C94D701969897988FEF30
:1003900093E090934B0080934A0080E293E0A3E9BE
:1003A000B0E08D939C930E941F0A0C94AB05E6ED80
:1003B000F8E10E943B0C11F00C94E801A3E9B0E0D5
:1003C0008D919C9190934B0080934A000C94AB05C7
:1003D000EAEDF8E10E943B0C11F00C94F9018FEF6B
:1003E00093E090934B0080934A00969897980C94D2
:1003F000AB05E0EEF8E10E943B0C11F00C94040216
:10040000969A979A0C94AB05E6EEF8E10E943B0CA5
:1004100011F00C940F02969897980C94AB05EAEEA5
:10042000F8E10E943B0C11F00C941C0288B390E19F
:10043000892788BB0C94AB05EEEEF8E10E943B0CDB
:1004400011F00C94290288B398E0892788BB0C949A
:10045000AB05E2EFF8E10E943B0C11F00C94540262
:10046000E8EFF8E10E94010BAAE8B0E038E00E9452
:10047000B60AAAE8B0E00E94DB0BA9E9B0E00C9351
:100480008091990080936400809199008093650029
:100490008091990080936600809199008093670015
:1004A000969897980C94AB05E8E0F9E10E943B0C14
:1004B00011F00C949202AAE8B0E038E00E94B60A6B
:1004C000AAE8B0E00E94DB0BA9E9B0E00C93A9E92F
:1004D000B0E00C9142E00E942B0C0C93009185003F
:1004E00040919900040FA4E6B0E00C9300918600BF
:1004F00040919900040FA5E6B0E00C9300918700AD
:1005000040919900040FA6E6B0E00C93009188009A
:1005100040919900040FA7E6B0E00C939698979845
:100520000C94AB05EEE0F9E10E943B0C11F00C9449
:10053000D002AAE8B0E038E00E94B60AAAE8B0E02B
:100540000E94DB0BA9E9B0E00C93A9E9B0E00C91A3
:1005500042E00E942B0C0C93009185004091990081
:10056000041BA4E6B0E00C93009186004091990032
:10057000041BA5E6B0E00C93009187004091990020
:10058000041BA6E6B0E00C9300918800409199000E
:10059000041BA7E6B0E00C93969897980C94AB05D3
:1005A000E4E1F9E10E943B0C11F00C94FB02009194
:1005B000850040918000041BA4E6B0E00C930091FC
:1005C000860040918000040FA5E6B0E00C930091F6
:1005D000870040918100041BA6E6B0E00C930091D7
:1005E000880040918100040FA7E6B0E00C93969A32
:1005F00097980C94AB05EAE1F9E10E943B0C11F0ED
:100600000C9426030091850040918000041BA4E611
:10061000B0E00C930091860040918000040FA5E6A5
:10062000B0E00C930091870040918100041BA6E686
:10063000B0E00C930091880040918100040FA7E680
:10064000B0E00C939698979A0C94AB05E0E2F9E130
:100650000E943B0C11F00C9476039698979A0091A7
:10066000850040918000041BA4E6B0E00C9300914B
:10067000860040918000040FA5E6B0E00C93009145
:10068000870040918100041BA6E6B0E00C93009126
:10069000880040918100040FA7E6B0E00C93AAE81F
:1006A000B0E038E00E94B60AAAE8B0E00E94DB0B96
:1006B000AFE3B1E00D931C9384E690E00E941E0B23
:1006C00080E293E090934B0080934A00AFE3B1E067
:1006D0008D919C910E941E0B8FEF93E090934B00A5
:1006E00080934A00969897980C94AB05E8E2F9E15C
:1006F0000E943B0C11F00C94C603969A97980091B7
:10070000850040918000041BA4E6B0E00C930091AA
:10071000860040918000040FA5E6B0E00C930091A4
:10072000870040918100041BA6E6B0E00C93009185
:10073000880040918100040FA7E6B0E00C93AAE87E
:10074000B0E038E00E94B60AAAE8B0E00E94DB0BF5
:10075000AFE3B1E00D931C9384E690E00E941E0B82
:1007600080E293E090934B0080934A00AFE3B1E0C6
:100770008D919C910E941E0B8FEF93E090934B0004
:1007800080934A00969897980C94AB05E0E3F9E1C2
:100790000E943B0C11F00C94FB03AAE8B0E038E097
:1007A0000E94B60AAAE8B0E00E94DB0BA3E4B1E025
:1007B0000C930091850040914301041BA4E6B0E036
:1007C0000C930091860040914301040FA5E6B0E030
:1007D0000C930091870040914301040FA6E6B0E01E
:1007E0000C930091880040914301041BA7E6B0E000
:1007F0000C930C94AB05E8E3F9E10E943B0C11F07B
:100800000C943004AAE8B0E038E00E94B60AAAE8E6
:10081000B0E00E94DB0BA3E4B1E00C9300918500F3
:1008200040914301040FA4E6B0E00C9300918600D0
:1008300040914301041BA5E6B0E00C9300918700B2
:1008400040914301041BA6E6B0E00C9300918800A0
:1008500040914301040FA7E6B0E00C930C94AB0564
:10086000E0E4F9E10E943B0C11F00C943B040E947F
:1008700019070C94AB05E6E4F9E10E943B0C11F07A
:100880000C946004ECE4F9E10E94010BA0E2B8E0F2
:10089000E2E8F0E00E94910B0E94F90A0E94080B26
:1008A000E6E5F9E10E94010BA0E2B8E0E4E8F0E03F
:1008B0000E94910B0E94F90A0E94080B0C94AB0550
:1008C000E0E6F9E10E943B0C11F00C946B040C94EF
:1008D000AF050C94AB05E6E6F9E10E943B0C11F084
:1008E0000C948C04AAE8B0E038E00E94B60AAAE8AA
:1008F000B0E00E94DB0BA1E4B1E00C930091410158
:10090000003218F011F00C9487040C948A0480E2F1
:10091000809341010C94AB05ECE6F9E10E943B0C9D
:1009200011F00C94F804E4E7F9E10E94010B07B11F
:10093000007E006007B90E942D0B082F192FA0E23E
:10094000B8E0E0E1F0E00E94820B0E94F90A0E9408
:10095000080BECE7F9E10E94010B07B1007E016092
:1009600007B90E942D0B082F192FA0E2B8E0E0E193
:10097000F0E00E94820B0E94F90A0E94080BE4E852
:10098000F9E10E94010B07B1007E026007B90E94E5
:100990002D0B082F192FA0E2B8E0E0E1F0E00E9453
:1009A000820B0E94F90A0E94080BECE8F9E10E9410
:1009B000010B07B1007E036007B90E942D0B082FC1
:1009C000192FA0E2B8E0E0E1F0E00E94820B0E9463
:1009D000F90A0E94080B82E390E00E941E0B0E941D
:1009E000CF0A082F013011F00C9493040C94AB053E
:1009F000E4E9F9E10E943B0C11F00C9403050C941E
:100A00003B090C94AB05ECE9F9E10E943B0C11F0B9
:100A10000C940E050C948B080C94AB05E4EAF9E1F8
:100A20000E943B0C11F00C94420580916800809369
:100A30004401809183008093680088EC90E00E94DC
:100A40001E0B07B1007E016007B90E942D0BA5E9BE
:100A5000B0E08D939C93809198008068809398007B
:100A6000EAEAF9E10E94010BA0E2B8E0E5E9F0E072
:100A70000E948A0B0E94F90A0E94080B0C94AD0593
:100A80000C94AB05EEEBF9E10E943B0C11F00C94D9
:100A90004D050C941C010C94AB05E6ECF9E10E94A9
:100AA0003B0C11F00C9458050C9493070C94AB0577
:100AB000EEECF9E10E943B0C11F00C9467058FEF0E
:100AC00093E090934B0080934A000C94AB05E0EDCB
:100AD000F9E10E943B0C11F00C949A05AAE8B0E0F1
:100AE00038E00E94B60AAAE8B0E00E94DB0BA8E654
:100AF000B0E00C9388EC90E00E941E0BE4EDF9E16D
:100B00000E94010B07B1007E016007B90E942D0B06
:100B1000082F192FA0E2B8E0E0E1F0E00E94820B7C
:100B20000E94F90AECEDF9E10E94010B0E94080B0A
:100B30000C94AB058FEF93E090934B0080934A00A9
:100B4000EEEDF9E10E94010B0E94080B80919800E4
:100B50008F77809398000C9489010C9489010091FF
:100B6000840040918200041BA5E4B1E00C93009145
:100B70004501409141010E942B0CA2E4B1E00C938D
:100B800000E213E0A1E4B1E04D9155270E949A0ADA
:100B9000A6E4B1E04D935C9381E0809345014091E0
:100BA000410100914501041718F011F00C947A06E8
:100BB00080E090E0ADE3B1E08D939C9380E0809382
:100BC000890000918900043018F011F00C940A0695
:100BD000ADE3B1E00D911C910F931F9307B1007E1F
:100BE000016007B90E942D0B482F592F1F910F91BB
:100BF000040F151FADE3B1E00D931C9384E190E069
:100C00000E941E0BA9E8B0E08C918F5F8C9310F4CA
:100C10000C94E105ADE3B1E00D911C9145E050E08D
:100C20000E949A0AA5E4B1E0AD90BB24A9E9B0E026
:100C3000AA0CBB1CAA0DBB1D4D935C9380E090E0F9
:100C4000ADE3B1E08D939C9380E0809389000091A7
:100C50008900043018F011F00C945006ADE3B1E0B7
:100C60000D911C910F931F9307B1007E026007B98D
:100C70000E942D0B482F592F1F910F91040F151F04
:100C8000ADE3B1E00D931C9384E190E00E941E0B54
:100C9000A9E8B0E08C918F5F8C9310F40C94270638
:100CA000ADE3B1E00D911C9145E050E00E949A0A3D
:100CB000A5E4B1E0AD90BB24A9EEB0E0AA0CBB1C4A
:100CC000AA0DBB1D4D935C930091680040914201B9
:100CD000040FA8E6B0E00C93A6E4B1E08D919C91DE
:100CE0000E941E0BA5E4B1E08C918F5F8C9310F4F1
:100CF0000C94CF05809184008093680084E690E096
:100D00000E941E0B80E090E0ADE3B1E08D939C93D8
:100D100080E08093890000918900043018F011F080
:100D20000C94B406ADE3B1E00D911C910F931F93A9
:100D300007B1007E016007B90E942D0B482F592F83
:100D40001F910F91040F151FADE3B1E00D931C939C
:100D500084E190E00E941E0BA9E8B0E08C918F5FC7
:100D60008C9310F40C948B06ADE3B1E00D911C91C3
:100D700045E050E00E949A0AA1E4B1E0AD90BB24A6
:100D8000A9E9B0E0AA0CBB1CAA0DBB1D4D935C9356
:100D900080E090E0ADE3B1E08D939C9380E08093A0
:100DA000890000918900043018F011F00C94FA06C3
:100DB000ADE3B1E00D911C910F931F9307B1007E3D
:100DC000026007B90E942D0B482F592F1F910F91D8
:100DD000040F151FADE3B1E00D931C9384E190E087
:100DE0000E941E0BA9E8B0E08C918F5F8C9310F4E9
:100DF0000C94D106ADE3B1E00D911C9145E050E0BB
:100E00000E949A0AA1E4B1E0AD90BB24A9EEB0E043
:100E1000AA0CBB1CAA0DBB1D4D935C938091820054
:100E2000809368000E942C0780E0809345010C9419
:100E30008901809185008093640080918600809371
:100E40006500809187008093660080918800809380
:100E50006700969897980895E2EEF9E10E94010BD9
:100E6000A0E2B8E0E1E4F1E00E94910B0E94F90AEF
:100E7000ECEDF9E10E94010B81E080934801409183
:100E8000410100914801041718F011F00C94640717
:100E9000A0E2B8E0E8E4F1E0A190BB24E9E9F0E0E9
:100EA000AA0CBB1CEA0DFB1D0E94820B0E94F90AD2
:100EB000ECEDF9E10E94010BA8E4B1E08C918F5FA9
:100EC0008C9310F40C943F0781E08093480140918B
:100ED000410100914801041718F011F00C948C079F
:100EE000A0E2B8E0E8E4F1E0A190BB24E9EEF0E094
:100EF000AA0CBB1CEA0DFB1D0E94820B0E94F90A82
:100F0000ECEDF9E10E94010BA8E4B1E08C918F5F58
:100F10008C9310F40C9467078DE00E940B0B0E94D9
:100F2000080B089508950E944F0CEAEEF9E10E9423
:100F3000010BA0E2B8E0E5E8F0E00E94910B0E940E
:100F4000F90AECE0FAE10E94010BA0E2B8E0E6E861
:100F5000F0E00E94910B0E94F90AECE0FAE10E9495
:100F6000010BA0E2B8E0E7E8F0E00E94910B0E94DC
:100F7000F90AECE0FAE10E94010BA0E2B8E0E8E82F
:100F8000F0E00E94910B0E94F90AEEE0FAE10E9463
:100F9000010B0E94080BE2E1FAE10E94010BAAE8B2
:100FA000B0E038E00E94B60AAAE8B0E0EAE2FAE16E
:100FB0000E943B0C11F40C94E407AAE8B0E00E94F4
:100FC000DB0BA5E8B0E00C93ECE2FAE10E94010B28
:100FD000AAE8B0E038E00E94B60AAAE8B0E0EAE287
:100FE000FAE10E943B0C11F40C94FD07AAE8B0E072
:100FF0000E94DB0BA6E8B0E00C93E4E4FAE10E9467
:10100000010BAAE8B0E038E00E94B60AAAE8B0E016
:10101000EAE2FAE10E943B0C11F40C941608AAE8EB
:10102000B0E00E94DB0BA7E8B0E00C93ECE5FAE13E
:101030000E94010BAAE8B0E038E00E94B60AAAE8D4
:10104000B0E0EAE2FAE10E943B0C11F40C942F08A4
:10105000AAE8B0E00E94DB0BA8E8B0E00C93809116
:101060008500809364008091860080936500809164
:101070008700809366008091880080936700E1E09C
:10108000F0E00E940F0BE4E7FAE10E94010BAAE8EE
:10109000B0E038E00E94B60AAAE8B0E0E2E8FAE17F
:1010A0000E943B0C11F00C947108E5E0F0E0A5E81B
:1010B000B0E07BE70E94100CE6E0F0E0A6E8B0E0CC
:1010C0007BE70E94100CE7E0F0E0A7E8B0E07BE7E8
:1010D0000E94100CE8E0F0E0A8E8B0E07BE70E9496
:1010E000100CE4E8FAE10E94010BAAE8B0E038E055
:1010F0000E94B60AAAE8B0E0EAE2FAE10E943B0CDC
:1011000011F00C9485080C941C010C94CB070E94E0
:10111000520C0C941C010E944F0CE2E9FAE10E946F
:10112000010BA0E2B8E0E0E8F0E00E94910B0E9421
:10113000F90AECE0FAE10E94010BA0E2B8E0E1E874
:10114000F0E00E94910B0E94F90AEEE0FAE10E94A1
:10115000010B0E94080BE6EBFAE10E94010BAAE8E2
:10116000B0E038E00E94B60AAAE8B0E0EAE2FAE1AC
:101170000E943B0C11F40C94C408AAE8B0E00E9451
:10118000DB0BA0E8B0E00C93ECECFAE10E94010B61
:10119000AAE8B0E038E00E94B60AAAE8B0E0EAE2C5
:1011A000FAE10E943B0C11F40C94DD08AAE8B0E0CF
:1011B0000E94DB0BA1E8B0E00C9300918500409108
:1011C0008000041BA4E6B0E00C93009186004091DF
:1011D0008000040FA5E6B0E00C93009187004091D9
:1011E0008100041BA6E6B0E00C93009188004091BA
:1011F0008100040FA7E6B0E00C93E1E0F0E00E946C
:101200000F0BE4E7FAE10E94010BAAE8B0E038E036
:101210000E94B60AAAE8B0E0E2E8FAE10E943B0CBC
:1012200011F00C942109E0E0F0E0A0E8B0E07BE7E9
:101230000E94100CE1E0F0E0A1E8B0E07BE70E9442
:10124000100CE4E8FAE10E94010BAAE8B0E038E0F3
:101250000E94B60AAAE8B0E0EAE2FAE10E943B0C7A
:1012600011F00C9435090C941C010C94AB080E94ED
:10127000520C0C941C010E944F0CE2EEFAE10E9409
:10128000010B0E94080BE6E0FBE10E94010BAAE8BB
:10129000B0E038E00E94B60AAAE8B0E0EAE2FAE17B
:1012A0000E943B0C11F40C945C09AAE8B0E00E9487
:1012B000DB0BA2E8B0E00C93E8E1FBE10E94010B3C
:1012C000AAE8B0E038E00E94B60AAAE8B0E0EAE294
:1012D000FAE10E943B0C11F40C947509AAE8B0E005
:1012E0000E94DB0BA3E8B0E00C93EAE2FBE10E9472
:1012F000010BAAE8B0E038E00E94B60AAAE8B0E024
:10130000EAE2FAE10E943B0C11F40C948E09AAE87F
:10131000B0E00E94DB0BA4E8B0E00C93ECE3FBE14F
:101320000E94010B0E94080BEEE4FBE10E94010BFE
:10133000A0E2B8E0E2E8F0E00E94910B0E94F90A16
:101340000E94080B8091820080936800E2E0F0E048
:101350000E940F0BE4E5FBE10E94010BA0E2B8E064
:10136000E3E8F0E00E94910B0E94F90A0E94080B4A
:101370008091830080936800E2E0F0E00E940F0B10
:10138000EAE5FBE10E94010BA0E2B8E0E4E8F0E04E
:101390000E94910B0E94F90A0E94080B8091840020
:1013A00080936800E2E0F0E00E940F0BE4E7FAE1CE
:1013B0000E94010BAAE8B0E038E00E94B60AAAE851
:1013C000B0E0E2E8FAE10E943B0C11F00C94FF0956
:1013D000E2E0F0E0A2E8B0E07BE70E94100CE3E07E
:1013E000F0E0A3E8B0E07BE70E94100CE4E0F0E05E
:1013F000A4E8B0E07BE70E94100C0C94150AE4E826
:10140000FAE10E94010BAAE8B0E038E00E94B60AB7
:10141000AAE8B0E0EAE2FAE10E943B0C11F00C9479
:10142000130A0C941C010C943D090E94520C0C945C
:101430001C01AAE9B0E08C918F5F8C930895809194
:101440008500809364008091860080936500809180
:1014500087008093660080918800809367000895DC
:1014600008950F921F922F923F924F925F927F9218
:10147000AF92BF920F931F932F933F934F935F931E
:101480006F937F938F939F93AF93BF93CF93DF938C
:10149000EF93FF938FB78F93A0E6B0E00E94700A9E
:1014A000E0E6FBE10E94010B8F918FBFFF91EF916E
:1014B000DF91CF91BF91AF919F918F917F916F916C
:1014C0005F914F913F912F911F910F91BF90AF90DE
:1014D0007F905F904F903F902F901F900F901895A6
:1014E000ED91FC91EF5FFF4FFC93EE93089500FCAC
:1014F00010D0089503D01ED001F8F9CF0024E8944D
:1015000057FF02C009D0689400F80BD010F80124EE
:10151000089502D009D00895509540954F5F5F4FD0
:101520000895E89417FF0895009510950F5F1F4FD9
:1015300068940895352F242FE894452B11F468946E
:101540000895512F402F0027112780E1440F551F88
:10155000001F111F021B130B416018F4020F131F11
:101560004E7F8A9599F70895A0E2B8E01ED08830A2
:1015700091F08D3039F03323C9F38D933A9563FEA2
:101580004AD0F4CF63FC04C08DE045D08AE043D05C
:1015900088278C9308953FD011973395E7CF80919A
:1015A0007F00882309F081E008950F929F93AF9305
:1015B000BF937F9380917F008823E1F3F89480911B
:1015C0007F008A9580937F0090917D00A9E6B0E02E
:1015D000A90F0024B01D8C919395943109F499279B
:1015E00090937D0078947F91BF91AF919F910F90E0
:1015F0000895A0E2B8E08D91882311F00CD0FBCFC4
:1016000008950E94360B802D11F005D0FACF089571
:101610008DE001D08AE05D9BFECF8CB9089588EE05
:1016200093E00CD03197D9F708953197F1F70895E9
:10163000689462F80895E89462F80895EF93FF9330
:10164000EE27E82BE92B31F0E0E0F2E13197F1F7FA
:101650000197D1F7FF91EF910895369A3699FECF11
:10166000369A3699FECF84B195B10895C8953196D2
:10167000002008957F930F93AF93BF938F939F9311
:101680008FB78F9380917F0004E1081B21F49CB1F8
:101690000E94180B12C000917E00A9E6B0E07727E7
:1016A0009CB1A00FB71F9C93839580937F000395F7
:1016B000043109F4002700937E008F918FBF9F9122
:1016C0008F91BF91AF910F917F9118956FB7F8945B
:1016D000882793E08D939A95E9F76FBF0895040FDB
:1016E000151F261F371F0895000F111F221F331FBC
:1016F000089500951095209530950F5F1F4F2F4F3F
:101700003F4F0895019110810EC0019111912191D7
:1017100030810BC00191108117FF05C03FEF2FEF03
:1017200004C0008111272227332737FF03C0E1DFE0
:101730008DE28D93CF93DF93CF92DF92EF92AA2425
:10174000BB24CC24DD24EE2440E2CAE0DD2755E0B2
:1017500093E38881890F87FD9F7083FD907F891BAC
:1017600089935A95A9F7C0DFAA1CBB1CCC1CDD1CB1
:10177000EE1C4A9551F7E894EFE0FF2782910ED0D6
:10178000EB30E0F71EF068948A2D0CD088278D93FB
:10179000EF90DF90CF90DF91CF910895982F8295B1
:1017A00001D0892F8F70805D26F0803309F4089571
:1017B00068948D93089500271127222733271DD081
:1017C0008A3328F4803318F005D015D0F9CF0EF401
:1017D00090CF089580538F93402F512F622F732FF6
:1017E00083DF82DF7CDF80DF8F919927080F191F4D
:1017F000291F391F08958D910895E894FCDF8032E8
:10180000E9F38B32D9F38930C9F38D3211F468943E
:10181000F2CF0895E199FECFEEBBFFBB319608955C
:1018200091E001C092E07B3751F47FB7F894F2DF8A
:101830008D918DBBE29AE19A9A95C9F77FBF772780
:10184000089591E001C092E0E5DFE09A8DB38D93B9
:101850009A95D1F70895FF93881BF9E0001FFA9538
:1018600011F4FF910895881F841B18F4840F889445
:10187000F5CF0894F3CF689401C0E894AF93BF9379
:101880008D9116F0919103C00E94360B902D89170F
:1018900018F011F48823A1F7BF91AF910895E8944F
:1018A00063F80895689463F80895696E6974000098
:1018B00048656C6C6F206174206261736963425289
:1018C00041214E5A2E007370656564006469720090
:1018D000726573657400676F000073746F70000049
:1018E0006261636B00006666000063616D0069728F
:1018F0000000616E676C6500616E676C6528312D54
:10190000323030293A2000006C656674000072693C
:10191000676874006C7475726E00727475726E0014
:1019200072767475726E00006C767475726E00005B
:101930006C6C7475726E0000726C7475726E00005F
:101940007A65726F000064756D70000073355F6DAD
:10195000696E3A20000073355F6D61783A200000AF
:101960007363616E00007373697A65006164636418
:10197000756D7000414443303A20000041444331CA
:101980003A200000414443323A20000041444333AE
:101990003A20000073636F6E6669670074636F6E50
:1019A00066696700747261636500747261636B6974
:1019B0006E672064697374616E63652000007265F0
:1019C000626F6F7400007A636F6E666967007800FB
:1019D0007368000073646973747C00007C00455276
:1019E000520066646973747C0000456E74657220F1
:1019F0007A65726F2076616C756520666F722073F0
:101A00006572766F7320286E6F7720002C00293A5C
:101A10000000736572766F203120286E20746F206D
:101A2000736B697029203E2000006E00736572762A
:101A30006F203220286E20746F20736B697029200C
:101A40003E200000736572766F203320286E20746C
:101A50006F20736B697029203E20000073657276D9
:101A60006F203420286E20746F20736B69702920DA
:101A70003E200000736176653F2028792F6E292073
:101A8000000079007265706561743F2028792F6EBF
:101A90002900456E746572207475726E2076616CD3
:101AA00075657320666F7220736572766F73202878
:101AB0006E6F772000006C5F7475726E20286E2048
:101AC000746F20736B697029203E2000725F7475FB
:101AD000726E20286E20746F20736B697029203E0F
:101AE0002000456E746572206D696E2C6D69642CE2
:101AF0006D61782076616C75657320666F722073F6
:101B00006572766F3A006D696E20286E20746F20C2
:101B10006E657874293A20006D696420286E2074FF
:101B20006F206E657874293A20006D617820286EE8
:101B300020746F206E657874293A20007465737480
:101B4000696E672073686172702E2E2E00006D69B9
:101B50006E2000006D69642000006D617820000037
:021B60002E0055
:00000001FF
